:020000040800F2
:10000000500A0020D9000008E1000008A101000802
:1000100000000000000000000000000000000000E0
:10002000000000000000000000000000E5000008E3
:1000300000000000000000001F010008230300086A
:10004000EB000008EB000008EB000008EB000008E4
:10005000EB000008EB000008EB000008EB000008D4
:10006000EB000008EB000008EB00000800000000B7
:10007000EB0000080000000000000000EB0000089A
:10008000EB000008EB000008EB000008EB000008A4
:10009000EB000008EB00000800000000EB00000887
:1000A000EB000008F5030008EB000008EB00000877
:1000B000EB000008EB000008EB000008EB00000874
:1000C0000448854600F016F9004800471903000867
:1000D000C046C046500A00200448804704480047F4
:1000E000FEE7FEE7FEE7FEE7FEE7FEE7D5030008D2
:1000F000C1000008EFF3108072B6704780F31088DB
:1001000070472A4A1368012B03D001231360284A41
:100110001060284A11602848284901607047EFF3B1
:10012000108272B62148016800291DD000210160AB
:100130001F48016800290AD0EFF3098120390068BF
:100140000160F0C144464D4656465F46F0C119492C
:1001500009680968F0C9F0B4F0C9A046A946B246DA
:10016000BB46F0BC81F3098882F31088042040422A
:100170000047104908600E49002008600B49012023
:1001800008600F480F490268114301600A480B4993
:1001900001600D480068006880F3088862B6704707
:1001A000EFF3098000B501F0DBFE00BD2400002064
:1001B0001C0000202000002004ED00E000000010E2
:1001C00020ED00E00000FFFF08ED00E030B50B4639
:1001D000014600202022012409E00D46D5409D4221
:1001E00005D31D469540491B2546954040191546A7
:1001F000521E002DF1DC30BD70B5002425460028CC
:1002000001DA01244042002901DA01254942FFF7C1
:10021000DDFFAC4200D04042002C00D0494270BD0E
:1002200003460B439B0703D009E008C9121F08C00F
:10023000042AFAD203E00B780370401C491C521EBA
:10024000F9D27047D2B201E00270401C491EFBD2C5
:1002500070470022F6E710B513460A4604461946D1
:10026000FFF7F0FF204610BD421E5378521C002BB2
:10027000FBD10B781370491C521C002BF9D170472D
:1002800010B5044605E00B780370401C002B00D02D
:10029000491C521EF7D2204610BD421C0178401C5A
:1002A0000029FBD1801A704730B504460020034670
:1002B00000E05B1C934203D2E05CCD5C401BF8D0B5
:1002C00030BD03460A780270401C491C002AF9D14F
:1002D0001846704730B505460020034600E05B1C19
:1002E000934205D2EC5CC85C201A01D1002CF6D1F7
:1002F00030BD0000064C0125064E05E0E36807CC42
:100300002B430C3C98471034B442F7D3FFF7DCFE84
:100310000C5900082C59000810B503F017FF0020F5
:1003200010BD10B501F0B2FE03F088FB01F0C6FE6F
:1003300010BD000070B5234CA2683820024022484E
:10034000082A34D001254300102A10D0182A0BD0D7
:10035000202A06D020682946C004800F8140184614
:1003600023E00120C00322E07D2000021FE0E168BD
:10037000C907C90F02D1002909D00020E168090688
:10038000CA0EE1684905490F002A02D002E018466A
:10039000F4E72022002900D108215043FFF716FF7F
:1003A000E16849038A0F29469140FFF70FFFA168D2
:1003B0001C2289091140054A5158FFF707FF0449DB
:1003C000086070BD0010024000127A0078520008E8
:1003D000F400002004490348886005490348086088
:1003E000704700000000000800ED00E00024F40069
:1003F000F400002070B50026F64301F047FE104DD2
:1004000020212868814318D12021284604F0CEF805
:10041000002812D034462021284604F0C7F80028CE
:1004200001D0686AC4B2601C04D0E1B2054802F091
:10043000BFFBEFE7044802F0C3FC01F03FFE70BDD4
:1004400000380140200600202C06002030B47446FD
:10045000641E2578641CAB4200D21D46635D5B00C0
:10046000E31830BC18470000002806D002060D49EA
:10047000120E03D0C0B2085C401C70470204120E7A
:1004800004D00004000E085C093070470202120E0E
:1004900004D00002000E085C11307047000E085CAA
:1004A000193070476F4E000802E008C8121F08C1DB
:1004B000002AFAD170477047002001E001C1121FE5
:1004C000002AFBD170470000F7B500268AB0054628
:1004D000002805D1FF223832274928A001F072FBFD
:1004E0000C98002807D1FF223932234924A001F0BB
:1004F00069FB00E0761CA85D202804D0092802D002
:100500000B988642F6D3002E33D01F48089600275A
:10051000B61D046813E006221CA12068FFF7DAFE6E
:1005200000280BD120682946801D089AFFF7D2FECB
:10053000002803D12068805D002818D00C341548AD
:1005400000688442E7D3002F13D020216846FFF7CC
:1005500080FE6A4628460B9901F04EF9002808D023
:100560006946B8470C99086000200DB0F0BDA76837
:10057000E9E70020C043F8E7B24B0008636D640070
:100580007265747000000000000000205F5F636D02
:10059000645F000004000020FEB5194604461430D4
:1005A000099F0A9E0B9D089B4060006020462262C6
:1005B00024308AC03A461846232101F032FFE16A0E
:1005C000A06A134B4218121F616A206A01F042FDB3
:1005D000E061202E04D3A7220E490FA001F0F2FA09
:1005E000214620318E754E7500206564A063A56498
:1005F00020630875A067E0670090019023462046BD
:100600000E4A19464C3003F043FB0020FEBD0000AB
:10061000D5340008815000087072696F726974796E
:10062000203C2052545F5448524541445F50524947
:100630004F524954595F4D4158000000F1380008AD
:1006400010B5029C6408640044720262C16100211A
:1006500043628162CA00121814325260491C12604F
:100660000129F7DB10BD70B505460024E0004019F4
:10067000143001F0C1FD641C012CF7DB70BD70B5B6
:100680000446FFF737FDA16F0546002901D020463B
:1006900088472846FFF732FD70BD10B500F052FCC8
:1006A000002010BD10B500F021FE002010BDFFB5E8
:1006B00083B01D4616460F460C9C01F0F3FC002843
:1006C00009D033463A46009501940020039904F07E
:1006D00069F807B0F0BD2B463246394600940398BE
:1006E00004F062F9F5E7000010B5114841692031C6
:1006F0004978890703D40F490020087015E0016983
:10070000002904D080220B48FFF7BAFD0DE001F06C
:1007100071F8002801D008A100E009A10548FFF701
:10072000D0FD09A10348FFF79FFD024810BD00005E
:1007300000000020F80000206D7368200000000019
:1007400066696E73682000003E00000070B50A4CB8
:1007500005466069002804D1A422084908A001F0D8
:1007600031FA6169FD22203148781040EA07920F82
:100770001043487070BD000000000020154C0008B8
:100780007368656C6C20213D2052545F4E554C4C73
:1007900000000000014A03C2704700000000002072
:1007A0007CB517491748FFF7F5FF83218900012021
:1007B00001F03CFA144D002868611BD00A21152075
:1007C0000123019100909B020022104910A002F029
:1007D0007FFD044600231A460FA1686902F0BAFAA9
:1007E0000120FFF7B3FF002C02D0204602F0E0FF0B
:1007F00000207CBD0AA001F09BFC0020C0437CBD12
:100800000C590008045800080000002039080008AE
:10081000747368656C6C0000736872780000000087
:100820006E6F206D656D6F727920666F72207368D0
:10083000656C6C0A00000000C24E01277069203010
:10084000417839434170FFF74FFF01F071FC0025FB
:1008500001F04AFB0400FBD470691B2C07D0014651
:1008600020310A78012A05D0022A0AD012E020306D
:100870000770EDE75B2C01D00D700BE002200870D3
:10088000E6E70D70412C43D0422C4AD0442C72D064
:10089000432C6DD0002CDBD0FF2CD9D0092C68D094
:1008A0007F2C67D0082CFCD00D2C74D00A2CFCD0E7
:1008B000C11DFF31FA31CA88502A00D3CD800B897F
:1008C000C9888B4268D2CA1A0146FF31FF30B7315E
:1008D000B8305918181801F08DFD41217069C90010
:1008E000095AFF30B7300C5470692121095CC907DF
:1008F00008D04121C900095AFF30B730091892A029
:1009000001F016FC7069FF30FF3002300489F4E01A
:10091000418C002903D0491E89B241840EE04584F0
:1009200096E7818C428C0B46491E8A4202DA521CA1
:10093000428402E0002B8BD04184418C50225143F1
:100940000918FF30B7302631FFF76AFC7069FF30B5
:10095000B730FFF7A2FC014670690246FF30FF3056
:100960000230C1800181104603F006FC70E702E00E
:1009700013E028E054E0FF30FF3002300089002807
:10098000CED072A001F0D4FB7069FF30FF3002308E
:100990000189491E15E088E0B7E0C11DFF31FA3139
:1009A0000A460989D2889142BAD2FF30B730095C31
:1009B00067A001F0BDFB7069FF30FF300230018994
:1009C000491C018144E7002403E060A001F0B0FB72
:1009D000641C7069FF30FF3002300089A042F4DCF3
:1009E00074695CA0FF34B73401F0A2FB00F002FF91
:1009F000012802D1204600F037FEFFF775FE0146C0
:100A0000224655A001F094FB7069FF30B730FFF724
:100A100044FC7169FF31FF310231C880088117E75A
:100A2000C21DFF32FA321389002B9FD0D1885B1E82
:100A3000491E89B29BB2D180138199422BD9CA1A1F
:100A40000146FF31FF30B831B7305918181801F09E
:100A5000D1FC43497069095AFF30B7300D54412128
:100A60007069C900095AFF30B73009183DA001F07C
:100A70005FFB7069FF30FF300230048903E033A070
:100A800001F056FB641C7069FF30FF300230C088F3
:100A9000A04297DBF3E735A001F04AFB30497069CB
:100AA000095AFF30B7300D54D2E603F0E5FB00F0F1
:100AB000A1FE01280ED1706920304078C00702D015
:100AC00024A001F035FB26497069095AFF30B73080
:100AD00000F020FEFFF708FE01F02AFB70695021AC
:100AE000FF30B730FFF7B5FB7069FF30FF300230E1
:100AF00024E016A001F01CFB641C7069FF30FF307D
:100B00000230C088A042F4DC0BE0FF30B7300C5458
:100B1000706920304078C00703D021460CA001F056
:100B200007FB7069FF30FF300230C188491C89B271
:100B3000C1800289521C02815029B5D3C58005812C
:100B400086E6000000000020257300000800000079
:100B5000256300000A0000002573257300000000D3
:100B60000602000008257320200800000820080065
:100B700010B501F097FA0028024801D0B83010BD36
:100B8000303010BDAC04002010B502A001F0D0FA46
:100B9000002010BD48656C6C6F2052542D54687253
:100BA000656164210A00000000B585B01421684623
:100BB000FFF74FFB0A490220CA6A0243CA6200BF1C
:100BC00000BF00BF0120800300900120019002902F
:100BD000002003906946034803F0CCFB05B000BD3C
:100BE000001002400004005070B50CA001F0A0FA03
:100BF0000F48104D04680CE002220FA12068FFF797
:100C000069FB002804D006CC0CA0083C01F090FA47
:100C10000C3428688442EFD3002070BD2D2D46751A
:100C20006E6374696F6E204C6973743A0A00000039
:100C300000000020040000205F5F0000252D3136F9
:100C400073202D2D2025730A00000000F0B591B00F
:100C500000262BA4082307AA042102A800F08CF880
:100C600008272246394628A001F062FA384600F0EB
:100C70002BFE2EA001F05CFA02A9304600F08CF8A1
:100C80000646002421E0A00007A90D580C3DFFF7FF
:100C900031FA297A6A464906127C490E914202D0FD
:100CA000FFF72CFA10E0FFF729FA284614300F90CE
:100CB00001F072FA002810D0E86900902B46082253
:100CC000394622A001F034FA641C0698A042DADC0E
:100CD000002ED1D1002011B0F0BD0F9801F071FAB3
:100CE000E969009101902B46082239461CA001F0C9
:100CF0001FFA0F9803F016FB0BA001F019FAE3E7B7
:100D00006576656E74000000252D2A2E7320202044
:100D10002020207365742020202073757370656E09
:100D200064207468726561640A00000020202D2D23
:100D30002D2D2D2D2D2D2D2D202D2D2D2D2D2D2DF0
:100D40002D2D2D2D2D2D2D0A00000000252D2A2EB4
:100D50002A73202030782530387820300A000000AF
:100D6000252D2A2E2A73202030782530387820250A
:100D70003033643A00000000F8B504461E461746BA
:100D80000D46084601F00CFE001D206025726760CC
:100D90000020E6602061F8BDF8B500260D460E6122
:100DA000C96800290CD0297A002909D02F680028A9
:100DB00008D00446FFF79EF90146002E05D010E04A
:100DC0000020F8BD3C460126F4E720460C38007AA6
:100DD0002A7A4006400E904203D00846FFF78EF96B
:100DE000EEE7686800262468BC4201D1002404E0D4
:100DF00010C0EA68761CB242F5D10846FFF77EF9CA
:100E000020462E61F8BD0000F0B591B000262FA459
:100E1000082308AA052103A8FFF7AEFF08272246EA
:100E200039462CA001F084F9384600F04DFD32A07F
:100E300001F07EF903A93046FFF7AEFF0646002514
:100E400027E0A80008A90C580C3CFFF753F9217AB9
:100E50006A464906127D490E914202D0FFF74EF9CB
:100E600016E0FFF74BF920461430109001F094F98A
:100E70000028109815D001F0A4F9218C628C009202
:100E80000191029023460822394622A001F050F930
:100E90006D1C0798A842D4DC002ECBD1002011B0E5
:100EA000F0BD01F08EF9218C628C009201910290CC
:100EB0002346082239461DA001F03AF9109803F0A4
:100EC00031FA19A001F034F9E2E700006D61696CB4
:100ED000626F7800252D2A2E7320656E747279203A
:100EE00073697A652073757370656E6420746872B7
:100EF0006561640A00000000202D2D2D2D20202D7D
:100F00002D2D2D202D2D2D2D2D2D2D2D2D2D2D2D1E
:100F10002D2D0A00252D2A2E2A73202530346420F9
:100F200020253034642025640A000000252D2A2E57
:100F30002A73202530346420202530346420256431
:100F40003A00000010B5074C07A0E16801F0F0F886
:100F50000AA0216901F0ECF80DA0616901F0E8F840
:100F600010BD000034000020746F74616C206D654A
:100F70006D6F72793A2025640A000000757365640C
:100F8000206D656D6F7279203A2025640A0000009B
:100F90006D6178696D756D20616C6C6F63617465EE
:100FA00064206D656D6F72793A2025640A00000037
:100FB000F0B591B000262DA4082307AA062102A8A7
:100FC000FFF7DAFE0827224639462BA001F0B0F8D9
:100FD000384600F079FC2FA001F0AAF802A93046AB
:100FE000FFF7DAFE0646002425E0A00007A90D5809
:100FF0000C3DFFF77FF8297A6A464906127C490EB4
:10100000914202D0FFF77AF814E0FFF777F828460C
:1010100014300F9001F0C0F800280F9813D001F0A1
:10102000D0F8A98C009101902B46082239461FA0C8
:1010300001F07EF8641C0698A042D6DC002ECDD1CB
:10104000002011B0F0BD01F0BCF8A98C0091019016
:101050002B46082239461AA001F06AF80F9803F0CF
:1010600061F91CA001F064F8E4E700006D7367719A
:101070007565756500000000252D2A2E7320656EAC
:101080007472792073757370656E6420746872650C
:1010900061640A00202D2D2D2D20202D2D2D2D2D8C
:1010A0002D2D2D2D2D2D2D2D2D0A0000252D2A2EF7
:1010B0002A732025303464202025640A00000000B3
:1010C000252D2A2E2A732025303464202025643AC9
:1010D000000000000A000000F0B591B0002623A433
:1010E000082309AA032104A8FFF746FE0827224681
:1010F000394620A001F01CF8384600F0E5FB26A098
:1011000001F016F804A93046FFF746FE0646002512
:1011100023E0A80009A90C580C3CFEF7EBFF217A4C
:101120006A464906127E490E914202D0FEF7E6FF5A
:1011300012E0FEF7E3FF2046143001F042F8E17FB1
:10114000226A082300930192029103902346082209
:10115000394619A000F0ECFF6D1C0898A842D8DCB5
:10116000002ECFD1002011B0F0BD00006D75746568
:1011700078000000252D2A2E732020206F776E65C1
:10118000722020686F6C642073757370656E6420C4
:101190007468726561640A00202D2D2D2D2D2D2D72
:1011A0002D202D2D2D2D202D2D2D2D2D2D2D2D2D89
:1011B0002D2D2D2D2D0A0000252D2A2E2A732025B8
:1011C0002D382E2A7320253034642025640A00002F
:1011D000F0B591B000262DA4082307AA022102A889
:1011E000FFF7CAFD0827224639462BA000F0A0FFD2
:1011F000384600F069FB2FA000F09AFF02A93046A4
:10120000FFF7CAFD0646002425E0A00007A90D58F7
:101210000C3DFEF76FFF297A6A464906127C490E9B
:10122000914202D0FEF76AFF14E0FEF767FF2846FE
:1012300014300F9000F0B0FF00280F9813D000F08A
:10124000C0FFA98B009101902B46082239461FA0B0
:1012500000F06EFF641C0698A042D6DC002ECDD1B3
:10126000002011B0F0BD00F0ACFFA98B00910190FF
:101270002B460822394619A000F05AFF0F9803F0B8
:1012800051F80BA000F054FFE4E7000073656D61B6
:1012900070686F7265000000252D2A2E732076205D
:1012A000202073757370656E642074687265616464
:1012B0000A000000202D2D2D202D2D2D2D2D2D2D22
:1012C0002D2D2D2D2D2D2D0A00000000252D2A2E2F
:1012D0002A7320253033642025640A00252D2A2E08
:1012E0002A7320253033642025643A00F0B5B1B06C
:1012F000002008903EA4082329AA012102A8FFF794
:101300003BFD08200146079022463B4800F010FFB5
:10131000079800F0D9FA39A000F00AFF02A908984E
:10132000FFF73AFD0025089059E0A80029A90C58BC
:101330000C3CFEF7DFFE0646207A69464006097C33
:10134000400E884203D03046FEF7D8FE46E08022A9
:10135000214609A8FEF764FF3046FEF7CFFE20467F
:1013600020300646407D00902346082233A007998E
:1013700000F0DEFE307D0007000F012808D00228B3
:1013800008D0002808D0042808D0032808D00AE094
:101390002DA006E02FA004E031A002E033A000E081
:1013A00035A000F0C5FEA06A064600E0401C0178AA
:1013B0002329FBD0E76A801B381A64214843394649
:1013C000FEF704FF0346216BA06C01910090E069D9
:1013D0003A46301AC1192BA000F0AAFE6D1C0698DF
:1013E000A842A2DC0898002898D131B0F0BD0000D6
:1013F000746872656164000098520008202D2D2DDC
:1014000020202D2D2D2D2D2D2D202D2D2D2D2D2D33
:101410002D2D2D2D202D2D2D2D2D2D2D2D2D2D2016
:10142000202D2D2D2D2D2D20202D2D2D2D2D2D2D13
:101430002D2D2D202D2D2D0A00000000252D2A2ECA
:101440002A7320253364200020726561647920208E
:10145000000000002073757370656E64000000006A
:1014600020696E69742020200000000020636C6FEA
:1014700073652020000000002072756E6E696E6733
:101480000000000020307825303878203078253072
:101490003878202020202530326425252020203057
:1014A000782530387820253033640A00F0B58FB0C5
:1014B000002626A4082307AA0A2102A8FFF75CFC3D
:1014C00008272246394623A000F032FE384600F0B5
:1014D000FBF92AA000F02CFE02A93046FFF75CFCC5
:1014E0000646002424E0A00007A90D580C3DFEF795
:1014F00001FE297A6A464906127C490E914202D0C1
:10150000FEF7FCFD13E0FEF7F9FDA96A686A019198
:1015100000902B460822394621A000F009FE687A87
:10152000C00701D024A000E026A000F001FE641C4A
:101530000698A042D7DC002ECED102F079FA0146FF
:1015400024A000F0F5FD00200FB0F0BD74696D65BA
:1015500072000000252D2A2E732020706572696F9D
:1015600064696320202074696D656F757420202084
:1015700020202020666C61670A000000202D2D2DA0
:101580002D2D2D2D2D2D2D202D2D2D2D2D2D2D2D98
:101590002D2D202D2D2D2D2D2D2D2D2D2D2D0A00D8
:1015A000252D2A2E2A73203078253038782030785F
:1015B00025303878200000006163746976617465B5
:1015C000640A000064656163746976617465640A25
:1015D0000000000063757272656E74207469636B3D
:1015E0003A3078253038780A00000000FFF7DCFA3E
:1015F0000FA3012216A1072003F0CAF90CA30122B0
:1016000013A1062003F0C4F909A3012210A10420AC
:1016100003F0BEF90124A4030F4D7D26F600AC6152
:10162000304602F037F8AC62304602F033F8F6E7A5
:1016300074657374204349553332204C3035312062
:1016400052542D546872656164210D0A0000000037
:101650006D61696E000000000004005010B500F0DC
:1016600001FBFFF7C3FF10BDF1B50098002500781E
:101670002E46002802D02248046834E000210846A3
:1016800000F07CF8F8BD06221EA12068FEF722FEBD
:10169000002827D127680098BF1DFEF7FEFD0246EF
:1016A00039460098FEF716FE00281BD1002D04D104
:1016B0003E463846FEF7F1FD05463946304601E024
:1016C000401C491C0278002A04D00B78002B01D062
:1016D0009A42F5D0801BA84200DA054639460BA095
:1016E00000F026FD0C340A4800688442CBD3002E5B
:1016F000C8D02A463146009801F0BEFCF8BD000073
:10170000000000205F5F636D645F000025730A00C6
:101710000400002038B5054601E0491E6D1C002973
:101720000CD028782028F8D00928F6D06A46284618
:10173000FEF7CAFE002803D02C4604E0002038BD86
:10174000009838BD641C2078202801D00028F9D1E9
:1017500000202070294603A000F0EAFC0020C043CE
:1017600038BD000025733A20636F6D6D616E642093
:101770006E6F7420666F756E642E0A0070B50EA0D1
:1017800000F0D6FC1348144D04680DE0062213A1A6
:101790002068FEF79FFD002805D106CC11A0891D09
:1017A000083C00F0C5FC0C3428688442EED310A03D
:1017B00000F0BEFC002070BD52542D54687265616B
:1017C00064207368656C6C20636F6D6D616E64730B
:1017D0003A0A000000000020040000205F5F636DF3
:1017E000645F0000252D313673202D2025730A00FB
:1017F0000A0000000120704770B5002315461C4602
:101800001E464AE00670401C5B1C0278202A01D06C
:10181000092A01D18B42F5D3082C10D321A000F066
:1018200087FC002605E0B000295826A000F080FCC7
:10183000761CA642F7D322A000F07AFC2FE08B4260
:101840002DD2D2B2222A03D0A200A850641C1BE0E1
:10185000A200401C5B1CA850641C08E05C2A04D158
:101860004278222A01D1401C5B1C401C5B1C027880
:10187000222A01D08B42F1D38B4210D20670401C39
:101880005B1C0AE0401C5B1C0278202A03D0092A5A
:1018900001D08B42F6D38B4201D28B42B5D3204686
:1018A00070BD0000546F6F206D616E7920617267AA
:1018B000732021205765206F6E6C79205573653A2F
:1018C0000A0000002573200010B5044602E003A0C2
:1018D00000F02EFC641EFAD210BD00002D000000A6
:1018E00010B50C48406800280DD000F0DBFB002844
:1018F0000AD101F015FF002806D006480021C9438F
:10190000083000F0A9FE10BDFEF7F4FB014980315C
:10191000486310BDAC04002010B50B484068002897
:101920000BD000F0BFFB002808D101F0F9FE002821
:1019300004D00548083000F0BFFD10BD02488030DB
:10194000406BFEF7DBFB10BDAC04002070B5214DF1
:1019500004462868844204D2A1221F491FA000F037
:1019600031F96868844204D3A2221B4923A000F005
:1019700029F96088002804D0A32217492AA000F082
:1019800021F9606829684018844210D04288002AF2
:101990000DD16A6890420AD0AA68824200D1AC6038
:1019A000426862604368621A084608301A50A068AC
:1019B0004018A0420CD04288002A09D1AA68A2424D
:1019C00000D1A86062684260401A626808315050D5
:1019D00070BD000034000020994F00082872745F29
:1019E00075696E74385F74202A296D656D203E3DDF
:1019F00020686561705F7074720000002872745F07
:101A000075696E74385F74202A296D656D203C20DD
:101A10002872745F75696E74385F74202A2968654E
:101A200061705F656E6400006D656D2D3E75736558
:101A300064203D3D20300000FFB589B004460E46CD
:101A400012A883C805900691780601D5484801E0A0
:101A5000474811380890F80601D57F087F00F8073D
:101A600001D0302000E02020079000200090B8072F
:101A70000DD5002A03DA2D205242009007E07807A6
:101A800001D52B2002E0380701D520200090002549
:101A9000002A04D130206946087101250CE00C9819
:101AA0000A2816D01107090F12090898415C01A8ED
:101AB00041556D1C002AF2D11398854200DD139523
:101AC000139905982022401A11213940002906D087
:101AD00014E010460A21FEF779FB0246E5E700997B
:101AE000002907D0002805DD401E03E0B44200D2E3
:101AF0002270641C0146401E0029F7DC0099002971
:101B000004D0B44200D22170401E641CF90605D5F1
:101B100008E0B44201D207992170641C0146401EBE
:101B20000029F6DC3023139F791E1391AF420ADDA2
:101B3000B44200D22370641CF5E7B44201D24B5D7D
:101B40002370641C00E001A92B466D1E002B07DDED
:101B5000069B002BF1D103E0B44200D22270641C3A
:101B60000146401E0029F7DC20460DB0F0BD000004
:101B7000804F00081CB514210A2001230191009018
:101B80005B020022074908A001F0A2FB040004D177
:101B9000C522074907A000F015F8204601F008FE0D
:101BA0001CBD00005D1600086D61696E000000003C
:101BB000494C000874696420213D2052545F4E5501
:101BC0004C4C000038B500236C462370084B5C6811
:101BD000002C01D0A04738BD13460A46014605A097
:101BE00000F0A6FA684600780028FBD038BD000057
:101BF0002C00002028257329206173736572746995
:101C00006F6E206661696C65642061742066756E14
:101C10006374696F6E3A25732C206C696E65206E53
:101C2000756D6265723A2564200A000070B54843FC
:101C3000044600F0EBFA050003D02246002100F034
:101C4000F0FB284670BD000070B5044C044D02E066
:101C500020688047241DAC42FAD370BDEC570008C1
:101C6000F457000870B5044C044D02E0206880472A
:101C7000241DAC42FAD370BDF45700080058000888
:101C800010B5FEF737FA034A5188491C5180FEF718
:101C900035FA10BDBC00002010B5FEF72BFA0A4C37
:101CA0006188491E09B26180002909DC0021618038
:101CB000FEF724FA6068002801D000F0ADFF10BDE7
:101CC000FEF71CFA10BD0000BC00002070B5040037
:101CD0006AD0FEF70FFA054600F0E4F9002809D0B3
:101CE000324933A000F024FA8B2292002F493AA007
:101CF000FFF768FF2846FEF701FAA00704D0374A2D
:101D00002A4937A0FFF75EFF414D2868844202D37D
:101D10006868844205D3314A2449521C3D48FFF784
:101D200051FF286884423FD3686884423CD2002136
:101D3000C94339480C3C01F08BF86088F5267601E0
:101D4000002802D02088B04211D034A000F0F0F971
:101D500023886288214638A000F0EAF960880028CC
:101D600005D11E4A114920323FA0FFF72BFF2088E2
:101D7000B04205D0194A0D4921323EA0FFF722FF9B
:101D8000002060802680A868844200D2AC60296868
:101D90006068611A401A2969081A28612046FFF70D
:101DA000D5FD1D4801F00CF870BD0000914F0008F2
:101DB00046756E6374696F6E5B25735D2073686131
:101DC0006C6C206E6F742062652075736564206989
:101DD0006E204953520A0000300000002E0200001D
:101DE00028282872745F75626173655F7429726D4B
:101DF000656D292026202852545F414C49474E5F8B
:101E000053495A45202D20312929203D3D203000BD
:101E100034000020B45300088C030020746F206647
:101E20007265652061206261642064617461206272
:101E30006C6F636B3A0A00006D656D3A203078254F
:101E40003038782C207573656420666C61673A20A1
:101E500025642C206D6167696320636F64653A2097
:101E60003078253034780A006D656D2D3E757365C8
:101E7000640000006D656D2D3E6D61676963203DF6
:101E80003D20484541505F4D414749430000000017
:101E900010B502F0C1FB0E487D21C9000068FEF7B5
:101EA00095F90C49401E884208D80B490B4A4861F5
:101EB000FF20D070002088610720086102F072F9CD
:101EC000FFF7C2FE0649074801F0EAF810BD00001E
:101ED000F4000020FFFFFF0000E000E020ED00E044
:101EE00000400020500A002038B5002069460870E4
:101EF000441E03E02146064800F0AAFF6946054853
:101F000000F0FCFD0128F5D16846007838BD0000DE
:101F10002C0600202006002070B504460D260F4D2B
:101F200011E00A2806D1AE628021284602F03EFB6D
:101F30000028F9D02078A8628021284602F036FBDC
:101F40000028F9D0641C20780028EAD140212846D6
:101F500002F02CFB0028F9D070BD000000380140D1
:101F60000446C16913A000F0E3F816A0A16900F0CF
:101F7000DFF818A0616900F0DBF81AA0216900F011
:101F8000D7F81CA0E16800F0D3F81EA0A16800F00B
:101F9000CFF820A0616800F0CBF822A0216800F003
:101FA000C7F82448016824A000F0C2F8FFF79EF9A2
:101FB000FEE700007073723A203078253038780AD6
:101FC000000000002070633A203078253038780A0D
:101FD00000000000206C723A203078253038780AF2
:101FE000000000007231323A203078253038780A0B
:101FF000000000007230333A203078253038780AFB
:10200000000000007230323A203078253038780AEB
:10201000000000007230313A203078253038780ADC
:10202000000000007230303A203078253038780ACD
:1020300000000000C00000206861726420666175C5
:102040006C74206F6E207468726561643A20257329
:102050000A000000F0B50646121DD008C000403846
:10206000094C074600229500521C4451102AFAD30D
:10207000016200214162816202463032C1624AC27D
:1020800001210906F963F0BDEFBEADDE10B5FEF724
:1020900031F8034A1178491C1170FEF72FF810BD72
:1020A0002800002010B5FEF725F803490C78FEF74C
:1020B00025F8204610BD00002800002010B5FEF7CE
:1020C00019F8034A1178491E1170FEF717F810BD70
:1020D0002800002010B50068143801F0E1FA002053
:1020E00010BDF8B5054614460E46084601F0BEFB85
:1020F00037461437002C15D0012C17D120362C6808
:102100000CE021212046727D095D14388A4204D2F8
:102110003946143000F039F802E02468AC42F0D1BE
:10212000AC4203D13946284600F02FF80020F8BD14
:102130000FB410B503AB7F210548029A01F0C4FE2D
:102140000348FFF7E9FE10BC08BC04B018470000C4
:102150000C03002010B5002801D0FFF7DDFE10BDF4
:102160000268516002680A60016048607047026856
:10217000516002680A6001604860704702685160FF
:1021800002680A60016048607047426811604268F6
:102190004A604160086070470168814201D10120B6
:1021A0007047002070470168814201D101207047CB
:1021B000002070470168814201D101207047002052
:1021C000704702460020114600E0401C0968914219
:1021D000FBD1704706C808384A6006C80838116045
:1021E00040600060704706C808384A6006C8083872
:1021F000116040600060704706C808384A6006C831
:10220000083811604060006070470000F8B50400B5
:102210001AD0FDF76FFF0546FFF744FF002809D0ED
:102220004E494FA0FFF784FFFF2219324B4956A0B9
:10223000FFF7C8FC2846FDF761FF544EE41CA508D3
:10224000F068AD00854201D90020F8BD0C2D00D208
:102250000C250021C9434E4800F0FAFDB0683168F2
:10226000F2688646401A9446531B70E00C18628848
:10227000002A6BD16268121A0C3AAA4266D36268CD
:10228000131A2A4618320C3B93422DD343190C33B0
:10229000F527CA187F0117800027578067685760A5
:1022A0009060012063606080506862460C3290420A
:1022B00002D00A4608328350306940190C30306130
:1022C0007269824200D27061F5204001208074451D
:1022D0001DD17268B0684388002B0DD090420BD09E
:1022E00040684018B060F6E7012060806068621ABC
:1022F000801A32698018E2E7904208D01804000C76
:1023000005D0FF228332154922A0FFF75BFC20484D
:1023100000F056FD601971680C30884205D9FF2223
:1023200087320E492548FFF74DFCA0070BD0FF224E
:1023300088320A492248FFF745FCFF2289320749C3
:1023400020A0FFF73FFC20460C30F8BD60688342B8
:102350008CD80F4800F034FD76E70000B84F000835
:1023600046756E6374696F6E5B25735D207368617B
:102370006C6C206E6F7420626520757365642069D3
:102380006E204953520A0000300000003400002043
:102390008C03002028286C66726565203D3D20680E
:1023A0006561705F656E6429207C7C2028216C66E5
:1023B0007265652D3E757365642929001054000807
:1023C0006853000828282872745F75626173655F1E
:1023D00074296D656D292026202852545F414C498F
:1023E000474E5F53495A45202D20312929203D3D34
:1023F0002030000010B5034681420FD28C189C4259
:102400000CD9811803E0641E2378491E0B70521EFC
:10241000F9D210BD0C781C70491C5B1C521EF9D2FD
:1024200010BD30B50346CCB2042A18D3810716D1AB
:102430002502194625432B042B4305E00B604B6016
:102440008B60CB601031103A102AF7D201E008C13E
:10245000121F042AFBD20B4601E01C705B1C521EAB
:10246000FBD230BD70B515460E46040004D10B4AB0
:102470000B490CA0FFF7A6FB32460321204600F0D3
:10248000B9FA20461430A06160610120A0830020C9
:10249000FF212062A177E077657270BD1D02000008
:1024A000D34C00086D7574657820213D2052545F2F
:1024B0004E554C4C00000000F8B5040005D1CB226D
:1024C0009200444944A0FFF77DFB204600F078FAD3
:1024D000032804D0454A3F494548FFF773FB0027CE
:1024E000FDF708FE009001F01BF9404D6D1D00281E
:1024F00008D138493FA0FFF71BFE2A4635494BA0BB
:10250000FFF760FBFDF7F6FD0646FFF7CBFD002861
:1025100008D0304946A0FFF70BFE2A462D4943A0BC
:10252000FFF750FB3046FDF7E9FD0098FDF7E6FDAB
:1025300001F0F6F80646FDF7DDFD0546206AB042DB
:1025400007D00024E44328463463FDF7D7FD204636
:10255000F8BDE17F491E0906090EE1772CD135212E
:10256000A27F095C8A4204D022461E32022100F07A
:1025700055FE204614300090FFF715FE0226F64364
:1025800000280AD0A08B310C88421ED2401CA083A8
:1025900000202062FF20A0770EE0606914382062DE
:1025A0002030407DA077E07FFF280ED2401CE077EE
:1025B0000098FFF78FFD01272846FDF79FFD002FAC
:1025C00001D000F029FB0020F8BD2846FDF796FD5C
:1025D0003046F8BD1F4D00086D7574657820213DAB
:1025E0002052545F4E554C4C000000002D0300005B
:1025F0002453000846756E6374696F6E5B25735DC6
:10260000207368616C6C206E6F7420626520757336
:102610006564206265666F726520736368656475C2
:102620006C65722073746172740A000030000000DF
:1026300046756E6374696F6E5B25735D20736861A8
:102640006C6C206E6F742062652075736564206900
:102650006E204953520A0000F3B581B00446FDF7DD
:1026600049FD064601F05CF85325ED00002808D12D
:10267000454946A0FFF75CFD2A46434951A0FFF7B4
:10268000A1FAFDF737FD0746FFF70CFD002808D03B
:102690003D494DA0FFF74CFD2A463B4949A0FFF7B5
:1026A00091FA3846FDF72AFD3046FDF727FD002C4C
:1026B00004D14F4A34494FA0FFF784FA204600F076
:1026C0007FF9032805D0A72292002F494E48FFF733
:1026D00079FA01F025F80546FDF70CFD06460020C5
:1026E00028630227206AFF43A84205D1E07FFF2824
:1026F0000CD2401CE07739E0A18B00290BD0491E99
:10270000A18325622035687DA077EFE73046FDF78D
:10271000F5FC3846FEBD029900292CD035214A5DD2
:10272000095C8A4204D22A463532022100F076FD45
:102730002046627A29461430FFF7D3FC029800281D
:1027400009DD28464C3002AA0021044601F0D2F9E6
:10275000204601F0C3FA3046FDF7D0FC00F05CFAE9
:10276000286B0028D6D1FDF7C5FC06463046FDF79C
:10277000C5FC0020FEBD0124E44330462C63FDF778
:10278000BDFC2046FEBD0000114D000846756E637D
:1027900074696F6E5B25735D207368616C6C206E6D
:1027A0006F742062652075736564206265666F7260
:1027B00065207363686564756C65722073746172FB
:1027C000740A00003000000046756E6374696F6E15
:1027D0005B25735D207368616C6C206E6F74206282
:1027E00065207573656420696E204953520A0000A4
:1027F0009B0200006D7574657820213D2052545F66
:102800004E554C4C0000000024530008F8B50F460C
:102810000646FDF76FFC0446FFF744FC002809D08C
:102820001A491BA0FFF784FCFF228732174922A018
:10283000FFF7C8F92046FDF761FC304600F0B0F81C
:10284000050005D1FF228B3210491CA0FFF7BAF911
:10285000E868FFF7DBFC041E17D00021EA68FFF7E9
:10286000E0FD26720020607208223946204600F002
:1028700003FCFDF73FFC064621460C31281DFFF7FF
:102880006FFC3046FDF73AFC2046F8BDED4F0008DE
:1028900046756E6374696F6E5B25735D2073686146
:1028A0006C6C206E6F74206265207573656420699E
:1028B0006E204953520A000030000000696E666FB6
:1028C000726D6174696F6E20213D2052545F4E55C8
:1028D0004C4C000070B5040005D1FF22BB320E49FC
:1028E0000EA0FFF76FF9207A000605D5FF22BC3253
:1028F00009490FA0FFF766F900202072FDF7FAFBE7
:10290000054620460C30FFF765FC2846FDF7F6FB30
:102910002046FFF7DBF970BD005000086F626A6562
:10292000637420213D2052545F4E554C4C000000F2
:1029300021286F626A6563742D3E74797065202664
:102940002052545F4F626A6563745F436C617373B6
:102950005F537461746963290000000070B504005E
:1029600005D1FF226732084908A0FFF72BF90020A4
:102970002072FDF7BFFB054620460C30FFF72AFC0E
:102980002846FDF7BBFB70BDDC4F00086F626A652F
:10299000637420213D2052545F4E554C4C00000082
:1029A000064A00210B01D35C834202D10801801842
:1029B0007047491C0729F5DB002070474C000020B8
:1029C00010B5040005D1FF22F032044904A0FFF73E
:1029D000F9F8207A4006400E10BD00002B50000888
:1029E0006F626A65637420213D2052545F4E554CDE
:1029F0004C000000F7B506460198FFF7D1FF05002F
:102A000005D1FF223432174917A0FFF7DBF8FFF793
:102A100037F92F1D6C680BE020460C3807D0B04208
:102A200005D1FF2244320F4915A0FFF7CBF82468E7
:102A3000BC42F1D1FFF730F9019880210843307290
:102A400008223046029900F017FBFDF753FB0446BD
:102A500031460C31281DFFF783FB2046FDF74EFB66
:102A6000FEBD0000CD4F0008696E666F726D617427
:102A7000696F6E20213D2052545F4E554C4C000032
:102A80006F626A20213D206F626A656374000000F6
:102A900010B5040005D1FF22DD32054905A0FFF77E
:102AA00091F8207A000601D5012010BD002010BD4C
:102AB000115000086F626A65637420213D205254F2
:102AC0005F4E554C4C00000010B58488C3886108E7
:102AD0005A0891420BD1E107DA07C90FD20F914290
:102AE00001D1002010BD01460820085E10BD8A42B9
:102AF00002D8891A0822825E501A10BD70B50D46A0
:102B0000040004D15B22104910A0FFF75BF82046B7
:102B1000FFF7DAFF002816D0A18820684908405C3A
:102B200028700822A088A25E4108521E914203D15B
:102B300001214840084004E0C007C00F491C49007B
:102B40000843A080012070BDE94B0008726220217B
:102B50003D2052545F4E554C4C00000070B5154658
:102B60000E46040004D1302209490AA0FFF72AF8D2
:102B7000002D04DC312206490AA0FFF723F80020CB
:102B8000A080E080A80880002660208170BD000041
:102B9000C04B0008726220213D2052545F4E554CBC
:102BA0004C00000073697A65203E20300000000070
:102BB00070B50D46040004D14122124912A0FFF75E
:102BC00001F82046FFF780FF0821615E884201D1AD
:102BD000002070BDE1882068490845540822E0883B
:102BE000A25E4108521E914203D101214840084093
:102BF00004E0C007C00F491C49000843E0800120E1
:102C000070BD0000D34B0008726220213D20525459
:102C10005F4E554C4C00000070B5FDF76BFA124C3E
:102C200005466088002815D1A068FDF71DFC401EF0
:102C30000E4AC10051586268143991420AD020707E
:102C40000B4861600078002808D010461C301C3109
:102C5000FDF757FA2846FDF751FA70BD10461C30B3
:102C60001C31FDF74EFAF5E7BC000020AC03002054
:102C70002800002070B5050005D1FF221832114947
:102C800011A0FEF79FFFFDF735FA024628462030D7
:102C9000017D2C4609090901491C0175407D0F4938
:102CA000C00041184868143404604868A8614C604A
:102CB00069610B49A86B8B68184388601046FDF763
:102CC0001DFA70BD4D500008746872656164202162
:102CD0003D2052545F4E554C4C000000AC03002088
:102CE000BC00002070B5050005D1FF224632114915
:102CF00011A0FEF767FFFDF7FDF92C4601461434DD
:102D000005CC083C426005CC083C1060646024603F
:102D10003520405D0D4AC00080180268824204D10F
:102D20000B48AB6B82689A4382600846FDF7E6F970
:102D300070BD0000675000087468726561642021EE
:102D40003D2052545F4E554C4C000000AC03002017
:102D5000BC000020F8B51E4615460F46040004D1FD
:102D6000D2220D490DA0FEF72DFF0120000485425F
:102D700004D3D32208490DA0FEF724FF3A460221CE
:102D80002046FFF737FE20461430A0616061A5831E
:102D900066720020F8BD0000734C000873656D205A
:102DA000213D2052545F4E554C4C000076616C75AD
:102DB00065203C2030783130303030550000000044
:102DC000F8B5040005D1FF22B8321A491AA0FEF75F
:102DD000F9FE2046FFF7F4FD022805D0FF22B932A4
:102DE00014491948FEF7EEFE0025FDF783F9064663
:102DF000204614300746FFF7D6F9002806D0A08BEE
:102E0000124988420FD2401CA08303E03846FFF7E6
:102E100061F901253046FDF771F9002D01D0FFF76A
:102E2000FBFE0020F8BD3046FDF768F90220C043E4
:102E3000F8BD0000B54C000873656D20213D20529F
:102E4000545F4E554C4C0000DC520008FFFF000060
:102E5000F3B581B0040005D1FF224D32374938A0C7
:102E6000FEF7B0FE2046FFF7ABFD022805D0FF229B
:102E70004E3232493648FEF7A5FEFDF73BF90646CD
:102E8000A08B002805D0401EA0833046FDF736F900
:102E900051E00298002809D0FDF72CF9009000F0CD
:102EA0003FFCFF256E35002806D00EE03046FDF7CA
:102EB00025F90120C043FEBD204926A0FFF738F9BF
:102EC0002A461E4931A0FEF77DFEFDF713F907469D
:102ED000FFF7E8F8002808D018492DA0FFF728F9D7
:102EE0002A46164929A0FEF76DFE3846FDF706F979
:102EF0000098FDF703F900F013FC05460020286355
:102F00002046627A29461430FFF7EBF80298002831
:102F100009DD28464C3002AA0021044600F0EAFDF3
:102F2000204600F0DBFE3046FDF7E8F8FFF774FEC0
:102F3000286B0028BFD10020FEBD0000A94C00086E
:102F400073656D20213D2052545F4E554C4C00005E
:102F5000DC52000846756E6374696F6E5B25735DA5
:102F6000207368616C6C206E6F74206265207573CD
:102F70006564206265666F72652073636865647559
:102F80006C65722073746172740A00003000000076
:102F900046756E6374696F6E5B25735D207368613F
:102FA0006C6C206E6F742062652075736564206997
:102FB0006E204953520A000008B509A0FFF7B8F87F
:102FC0000AA0FFF7B5F812A0009005230122032103
:102FD00012A0FFF7ADF819A0FFF7AAF808BD00008E
:102FE0000A205C207C202F0A000000002D20525473
:102FF000202D2020202020546872656164204F70AD
:1030000065726174696E672053797374656D0A0027
:10301000417567203230203230323400202F207C3E
:10302000205C202020202025642E25642E2564206D
:103030006275696C642025730A000000203230300C
:1030400036202D203230323020436F70797269671C
:1030500068742062792072742D74687265616420CE
:103060007465616D0A000000014600E0491C0A78A1
:10307000002AFBD1081A704710B5002A08D0034671
:103080000C781C70491C5B1C002C05D0521EF7D11B
:1030900010BD19705B1C00E00021521EF9D110BD5B
:1030A000F8B50646C01C84088D080F46A400AD0084
:1030B000FDF720F80090FEF7F5FF002808D01A4928
:1030C0001AA0FFF735F8D222174922A0FEF77AFDA1
:1030D0000098FDF713F8182D1FD928461838A0427C
:1030E0001BD3291B1C4D18392C60F522E9605201B5
:1030F00022800C3100206160A06060800819686047
:1031000002800122428041608160002313A11548A2
:10311000FFF720FE2868A860F8BD3A46314612A0A5
:10312000FFF706F8F8BD0000A44F000846756E636F
:1031300074696F6E5B25735D207368616C6C206EC3
:103140006F74206265207573656420696E20495331
:10315000520A0000300000003400002068656170F1
:10316000000000008C0300206D656D20696E69749D
:103170002C206572726F7220626567696E206164CF
:10318000647265737320307825782C20616E64201A
:10319000656E64206164647265737320307825788D
:1031A0000A00000010B50023094A0A4C5380184653
:1031B000C10009194960401C09602028F8DB1F2064
:1031C0001070034853600C3093604060006010BD85
:1031D000BC000020AC03002010B5074CA068FDF730
:1031E00043F9401E0549C0000858143860601C307F
:1031F000FCF7BFFF10BD0000BC000020AC030020A6
:10320000044A0020C100891849600960401CF9D0B7
:1032100070470000D400002070470000F8B5164643
:103220000D46040004D1224A224923A0FEF7CAFC1D
:103230002046FFF7C5FB012805D04F22D2001D49CB
:103240002248FEF7BFFC002D22D0012D24D0022DF4
:1032500011D1FCF74FFF254620350090287D01272E
:103260000007000F012808D0307868758740A763F1
:103270000098FCF743FF0020F8BD2046FFF732FD21
:103280003078687587402046A763FFF7F3FCEFE7C7
:10329000204600F08DFAF8BD2046FFF7F9FB012823
:1032A000204602D000F034F8F8BD00F0A1F8F8BDD7
:1032B00077020000FA50000874687265616420218A
:1032C0003D2052545F4E554C4C00000054540008B1
:1032D000FFB585B01D4601200E9F0F9E0599FFF793
:1032E00095FA041E0DD02846FEF790FF00280AD05C
:1032F00069460396A1C105A90EC92046FDF74CF900
:10330000204609B0F0BD2046FFF7E4FA0020F8E7B8
:1033100070B5040005D1FF229F321E491EA0FEF7A2
:1033200051FC2046FFF74CFB012805D0FF22A032BC
:1033300018491E48FEF746FC2046FFF7A9FB002867
:1033400005D0FF22A132134919A0FEF73BFC254608
:103350002035287D0107090F042918D0000702D065
:103360002046FFF7BFFC2046FDF789F920464C3088
:1033700000F020FCFCF7BEFE06460420287521461E
:1033800014311A48FEF7F3FE3046FCF7B7FE002072
:1033900070BD0000C350000874687265616420212C
:1033A0003D2052545F4E554C4C00000054540008D0
:1033B00072745F6F626A6563745F69735F73797358
:1033C00074656D6F626A656374282872745F6F62DA
:1033D0006A6563745F742974687265616429203D4D
:1033E0003D2052545F46414C53450000C800002028
:1033F00070B5040005D1FF223A32224922A0FEF71F
:10340000E1FB2046FFF7DCFA012805D0FF223B3222
:103410001C492248FEF7D6FB2046FFF739FB00285F
:1034200005D1FF223C3217491DA0FEF7CBFB2546F4
:103430002035287D0107090F04291DD0000702D07F
:103440002046FFF74FFC2046FDF719F920464C3087
:1034500000F0B0FB042028752046FFF719FB012877
:103460000CD0FCF747FE0546214614311848FEF7FC
:103470007EFE2846FCF742FE002070BD2046FFF786
:103480006DFAF9E7B2500008746872656164202132
:103490003D2052545F4E554C4C00000054540008DF
:1034A00072745F6F626A6563745F69735F73797367
:1034B00074656D6F626A656374282872745F6F62E9
:1034C0006A6563745F7429746872656164290000B9
:1034D000C800002070B513480468FCF70BFE0546D1
:1034E0002046FDF7CCF82046FFF7FCFB04213420F2
:1034F000015520464C3000F05DFB2046FFF7C8FA2E
:1035000001280AD0214614310748FEF730FEFFF7A4
:1035100083FB2846FCF7F2FD70BD2046FFF71EFA3C
:10352000F5E70000C0000020C8000020064D002480
:10353000A0002858002800D08047641C042CF7D332
:1035400000F004F8F3E70000FC02002070B5FCF77F
:10355000D1FD0446FEF7A6FD002808D0154916A0A7
:10356000FEF7E6FD932213491DA0FEF72BFB204634
:1035700012E01C4801680C4605C90839426005C9BB
:10358000083910604960143C0960A06AFEF79EFB90
:103590002046FFF79FF92846FCF7B0FDFCF7AAFD8F
:1035A0000546104801688142E3D12846FCF7A6FD94
:1035B00070BD00005D4C000846756E6374696F6EE7
:1035C0005B25735D207368616C6C206E6F74206284
:1035D00065207573656420696E204953520A0000A6
:1035E00030000000C80000201FB5202307481F221C
:1035F000D9006C460FC40023054A06A1803800F0AC
:103600000DF80248803800F0D3F81FBDFC010020FF
:103610002D3500087469646C65000000FFB585B045
:10362000109E119D0E9C070004D1E9220D490EA0A9
:10363000FEF7C8FA002C04D1EA220A490FA0FEF7CF
:10364000C1FA01213846069AFFF7D4F90F98019084
:1036500002960395009406A90EC93846FCF79CFF14
:1036600009B0F0BD91500008746872656164202152
:103670003D2052545F4E554C4C0000007374616302
:103680006B5F737461727420213D2052545F4E55FC
:103690004C4C000010B500F0B5F900F047F810BD33
:1036A00070B5040004D1164A164917A0FEF78AFA2D
:1036B0002046FFF785F9012805D05F22D200114985
:1036C0001648FEF77FFA3420005D0007000F02283D
:1036D00002D00020C04370BDFCF70CFD054620461B
:1036E0001430FEF780FD20464C3000F099FB284650
:1036F000FCF704FD2046FFF7BDFA002070BD000076
:10370000F70200001E510008746872656164202190
:103710003D2052545F4E554C4C000000545400085C
:103720000148006870470000C0000020F1B5FCF7B8
:10373000E1FC054616480468002C05D1FF22FC3246
:10374000144915A0FEF73EFA2046FFF739F9012883
:1037500005D0FF22FD320F491448FEF733FA204608
:1037600000F084F820464C306A460021064600F0FE
:10377000C1F9304600F0B2FA2846FCF7BFFCFFF76B
:103780004BFA206B801C00D120630020F8BD0000A4
:10379000C0000020D4500008746872656164202164
:1037A0003D2052545F4E554C4C00000054540008CC
:1037B00070B5050005D1FF220E32164916A0FEF79E
:1037C00001FA2C462034207D000705D0FF220F325D
:1037D000104916A0FEF7F6F92846FFF7F1F8012880
:1037E00005D0FF2210320B491E48FEF7EBF9A07DF1
:1037F0000121607581400220A96320752846FFF7EA
:103800004FFF19480068002801D0FFF705FA002093
:1038100070BD0000A05000087468726561642021CA
:103820003D2052545F4E554C4C0000002874687285
:103830006561642D3E7374617420262052545F5478
:1038400048524541445F535441545F4D41534B29C5
:10385000203D3D2052545F5448524541445F494EFB
:103860004954000054540008C000002070B5040002
:1038700004D1174A174918A0FEF7A4F92046FFF70C
:103880009FF8012805D0124A1249521C1748FEF72A
:1038900099F925462035287D0007000F012802D020
:1038A0000020C04370BDFCF725FC06462046FFF70C
:1038B00019FA287D00090001801C287520464C302B
:1038C00000F0AEFA3046FCF719FC002070BD000095
:1038D000CD0200000C5100087468726561642021FB
:1038E0003D2052545F4E554C4C000000545400088B
:1038F00010B5040004D1144A144915A0FEF762F96A
:103900003420005D0007000F022805D0C922920074
:103910000E4914A0FEF756F92046FFF751F801288A
:1039200005D0094A0949921C1D48FEF74BF90120B0
:10393000C043206320461430FEF755FC2046FFF7B5
:1039400099F9FFF769F910BD230300002F51000812
:1039500074687265616420213D2052545F4E554C5D
:103960004C000000287468726561642D3E737461B8
:103970007420262052545F5448524541445F5354AA
:1039800041545F4D41534B29203D3D2052545F54DB
:1039900048524541445F53555350454E4400000042
:1039A0005454000870B5FCF7A5FB054613480068A1
:1039B000014620310E46097D0907090F012917D15B
:1039C00082694169914213D014300446FEF70BFC22
:1039D000707D0B49C000401841680C60416861600F
:1039E000446020602846FCF789FBFFF715F902E0E8
:1039F0002846FCF783FB002070BD0000C0000020BB
:103A0000AC03002070B5002802DA0020C04370BD6E
:103A10007D25ED002946FCF7EFFB2A46044651437D
:103A2000501E081854432946FCF7E6FB001970BDE8
:103A300001480068704700001800002010B50848D1
:103A40000168491C0160FFF76BFE816C491E8164AF
:103A500003D1416C8164FFF7A5FF00F003F810BDAE
:103A600018000020FEB5684601900090FFF7E0FFC7
:103A70000646FCF73FFB05462FE01C481C4904683E
:103A80006069143C301A88422CD22046FCF7EBFDCA
:103A9000607A810702D440084000607221461431E8
:103AA0000F466846FEF76AFBE169206A8847FFF720
:103AB000BFFF06466846FEF77DFB00280DD138465D
:103AC000FEF79AFB607A810707D5C10705D0400849
:103AD00040006072204600F001F90448FEF76AFBDE
:103AE0000028CAD02846FCF709FBFEBDD400002000
:103AF000FFFFFF7F70B515460E46040005D1FF227B
:103B0000DA32174917A0FEF75DF82046FEF758FF96
:103B10000A2805D0FF22DB32114917A0FEF752F820
:103B2000FCF7E8FA3300FCF791FC050604090D12D6
:103B30001700616A0FE0296861620DE0617AFD2279
:103B4000114002E0617A02221143617204E0617A5D
:103B5000C90700D001212960FCF7D0FA002070BD10
:103B60008C51000874696D657220213D2052545FAC
:103B70004E554C4C0000000072745F6F626A6563C2
:103B8000745F6765745F74797065282674696D6504
:103B9000722D3E706172656E7429203D3D20525435
:103BA0005F4F626A6563745F436C6173735F5469EE
:103BB0006D65720070B5040004D1DD22144915A0B2
:103BC000FEF700F82046FEF7FBFE0A2804D0DE22AE
:103BD0000F4915A0FDF7F6FF2046FEF759FF002814
:103BE00004D1DF220A491FA0FDF7ECFFFCF782FA9F
:103BF00005462046FCF737FD607A400840006072B9
:103C00002846FCF77BFA2046FEF7A8FE002070BD90
:103C10004F51000874696D657220213D2052545F38
:103C20004E554C4C0000000072745F6F626A656311
:103C3000745F6765745F74797065282674696D6553
:103C4000722D3E706172656E7429203D3D20525484
:103C50005F4F626A6563745F436C6173735F54693D
:103C60006D65720072745F6F626A6563745F697319
:103C70005F73797374656D6F626A65637428267407
:103C8000696D65722D3E706172656E742900000069
:103C9000FFB581B00B9D1E460F46040004D1C9221A
:103CA000084909A0FDF78EFF3A460A212046FEF793
:103CB000A1FE0095324620460A9B0399FCF7C0FC02
:103CC00005B0F0BD4151000874696D657220213D59
:103CD0002052545F4E554C4C00000000FEB50400CD
:103CE00005D1FF2242322E492EA0FDF76BFF204660
:103CF000FEF766FE0A2805D0FF22433228492EA08F
:103D0000FDF760FFFCF7F6F902902046FCF7ABFCEC
:103D1000607A4008400060723648616A814205D38B
:103D2000FF2252321E4934A0FDF74CFFFFF780FE00
:103D3000616A6D4643183948A362864600220090A6
:103D40000CE00768019EBC46BE1B76699E4203D00C
:103D5000F71A284EB74209D3604668509100685858
:103D6000D600019676447668B042EAD1002A02D0A5
:103D7000491908304860521CF0D02848001F0168DB
:103D8000491C0160214614310098FEF7F7F9607A6A
:103D90000121084360720298FCF7B0F90020FEBDD3
:103DA0006F51000874696D657220213D2052545F87
:103DB0004E554C4C0000000072745F6F626A656380
:103DC000745F6765745F74797065282674696D65C2
:103DD000722D3E706172656E7429203D3D205254F3
:103DE0005F4F626A6563745F436C6173735F5469AC
:103DF0006D657200FFFFFF7F74696D65722D3E690E
:103E00006E69745F7469636B203C2052545F54493F
:103E1000434B5F4D4158202F20320000D40000203A
:103E200070B5040005D1FF22B732124912A0FDF788
:103E3000C9FE2046FEF7C4FD0A2805D0FF22B8328D
:103E40000C4912A0FDF7BEFE607AC0070ED0FCF749
:103E500051F905462046FCF706FC607A4008400010
:103E600060722846FCF74AF9002070BD0020C0436C
:103E700070BD00007E51000874696D657220213D9F
:103E80002052545F4E554C4C0000000072745F6F1E
:103E9000626A6563745F6765745F7479706528260C
:103EA00074696D65722D3E706172656E7429203D76
:103EB0003D2052545F4F626A6563745F436C617367
:103EC000735F54696D657200FFB585B0059C0698F7
:103ED0001F4620180390A04204D20020C043039044
:103EE000001B069008E1252804D003998C427ED25D
:103EF00020707CE000250423082610220799491C25
:103F0000079108782D2812D02B2812D0202812D003
:103F1000232812D0302812D00B780026F643303BED
:103F20000A2B0FD207A800F015FA064613E0154336
:103F3000E4E71D43E2E73543E0E7202000E001200D
:103F40000543DBE72A2806D1491C079140CF002E04
:103F500001DA76421543079800230178DB432E29C6
:103F600013D1401C079001780A46303A0A2A04D23D
:103F700007A800F0EFF9034604E02A2904D1401C09
:103F8000079008CF002B00DA002307990022087859
:103F9000682801D06C2802D1491C02460791097893
:103FA0000A206F2977D00CDC632922D004DC252974
:103FB00072D058290DD188E0642901D0692908D12F
:103FC00087E070296AD0732930D0752973D0782999
:103FD0007DD00398844201D2252020700798641C6C
:103FE0000178002969D00398844200D22170641CB2
:103FF0007FE0E80609D42020761E002E05DD039917
:104000008C4200D22070641CF6E7387803993F1D7B
:104010008C4200D22070202003E003998C4200D211
:104020002070641C761E002EF7DC62E002CF0029AF
:1040300000D140A1002000E0401CB04202D00A5C48
:10404000002AF9D1002B02DD984200DD1846EA066D
:104050000AD420223346761E834205DD039B9C4210
:1040600000D22270641CF5E7002207E0039B9C420B
:1040700001D20B782370491C521C641C8242F5DB70
:1040800020213246761E824233DD039A944200D2CA
:104090002170641CF5E716E010E0FFE7701C02D108
:1040A00008260120054301930096029504CF1023B2
:1040B000204603991AE00EE009E02BE003988442C1
:1040C00095D2252014E7082005E040200543102064
:1040D00001E002210D436C2A01D0682A1DD004CFD3
:1040E000019303460096029520460399FDF7A4FC30
:1040F00004460798401C079007980078002800D0D5
:10410000F1E60698002811D0039900208C420BD2CA
:1041100020700BE0401E0790EBE739883F1D8AB204
:10412000A907DDD512B2DBE72039C877059809B0B9
:10413000201AF0BD284E554C4C2900000020704735
:1041400000207047002070470020704710B5FBF733
:10415000D1FFFDF79DFEFEF72FFFFFF751F8FFF7A8
:1041600021F8FDF707FDFFF757F8FFF73DFAFFF7D6
:1041700033F8002010BD000010B5044606A0FDF77E
:10418000D7FFFCF7B1FA22460146FF32B7320448A6
:10419000FDF7CEFF002010BD1B5B324B0D00000071
:1041A000580B0008F0B52C4910228DB08818FEF786
:1041B000D5FC294800231A4628A11C30FEF7CAFD69
:1041C000142107A8FCF745F81C216846FCF741F8C4
:1041D000254F0120F96A0143F96200BF00BF00BF0B
:1041E0000320C0020790022001250890002405202A
:1041F000099507A90B950A94000700F0BBF8B86B66
:10420000AE033043B86300BF00BF00BFE1204002EF
:10421000039404940594069402900C20134C00908F
:104220006946204600F0C9F9002800D0FEE7206862
:104230002843206021682020014321600C49086840
:10424000FF221202904330430860012009494006D2
:1042500008600DB0F0BD0000100600207368656CAA
:104260006C5F7278000000000010024000380140CE
:1042700018E400E000E100E0F8B5C61DFF36044692
:10428000FA36F088002849D02746A08CFF37B73788
:10429000052823D33846502239465038FCF704F815
:1042A00000283BD000255020684300190146763194
:1042B00050222630FBF7B4FF6D1C042DF3DB502099
:1042C00045432819263005465021FBF7C2FFF288E6
:1042D00028463946FBF7A4FF05201EE0002809D038
:1042E0005021484300190A4639462A38FBF7DCFFBB
:1042F000002813D0A08C6084502148430019263038
:10430000FBF7A7FFA08C502148430019F2883946DB
:104310002630FBF785FFA08C401CA084A08C608415
:10432000F8BD000070B5054604680BE0214614395D
:1043300006A0FDF7FDFE2068A84202D004A0FDF70C
:10434000F7FE2468AC42F1D170BD00002573000077
:104350002F0000000246002006E04B1C13600A23D9
:10436000097858433038081811680B78303B0A2B0D
:10437000F3D37047F8B50C46074600251BE0012033
:10438000A840064016D031463846626800F03FF833
:1043900031463846A26800F044F86068022809D126
:1043A0002269FF2E3146384602D800F015F801E0A8
:1043B00000F01FF86D1C26683046E840DFD16068C9
:1043C000012801D0022806D1E1687A68304682438C
:1043D000484302437A60F8BD10B5046A0B464B436C
:1043E0004B434B431901C91A8C4353431C4304628A
:1043F00010BD0B0A19465943594310B559430B01D7
:104400005C1A436A5143A3430B43436210BD10B58A
:10441000036849434C000C19A34351430B43036009
:1044200010BD10B5C36849434C000C19A343514358
:104430000B43C36010BD000010B500F04BF80349FA
:1044400089684905490FC84010BD000000100240AE
:1044500010B5FFF7F1FF044989684904490F0329A2
:1044600001D3C91EC84010BD0010024010B5FFF7AF
:10447000E3FF044989684903490F032901D3C91E91
:10448000C84010BD0010024010B50F4CE068C007D6
:10449000C00F01D00D4800E00D48E1680906CA0EC2
:1044A000E1684905490F002A00D12022002900D1E6
:1044B00008215043FBF78AFEE16849038A0F012176
:1044C0009140FBF783FE10BD0010024000127A00FD
:1044D0000024F40010B510498868382210400828DC
:1044E0000ED010280ED018280FD0202810D0086821
:1044F0000121C004800F81400848FBF767FE10BD12
:10450000074810BDFFF7C0FF10BD7D20000210BDA1
:104510000120C00310BD0000001002400024F40080
:1045200000127A0070B504461B480D46844202D141
:10453000FFF79CFF16E01948844201D1012000E0FA
:10454000002017498C4201D1012100E000210843DD
:1045500014498C4201D1012100E00021084319D007
:10456000FFF776FF22680123DB031A4069089A42AD
:1045700002D14000401802E0002A0BD10818294659
:10458000FBF724FE0146084A1039914202D8E06048
:10459000002070BD012070BD003801400044004083
:1045A00000480040004C0040EFFF0000C06981431C
:1045B00001D0002070470120704710B5CA68036819
:1045C00001242403A343134303600A6943680324BB
:1045D0002403A343134343604A6803680124E403AC
:1045E000A343134303600A6803680C24A3431343E3
:1045F00003604A690368E401A343134303608A69C3
:1046000083686410A343134383608968FFF78AFFBC
:10461000002800D0012010BD10B5214902200A68F1
:104620009208920002430A601E48016882151143F5
:1046300001600168C9434905C917491CF9D0C1681F
:10464000194A1140194A1143C1600168012212063A
:10465000114301600168C9438901C917491CF9D098
:10466000C168012212041143C16082680221D2088C
:10467000D2000A4382603822816811401029FBD1A0
:10468000816807221202914381608168120191437F
:1046900081608168120191438160FBF74BFE10BD80
:1046A000002002400010024006F8F9FF60020200FC
:1046B00070B515460E46040004D1204A204921A0B9
:1046C000FDF780FA002E05D11C4A1D49521C1FA07F
:1046D000FDF778FA1F480068002805D1174A1849E5
:1046E000921C1DA0FDF76EFA6069002805D1134ADF
:1046F0001349D21C1CA0FDF765FA2369002B01D0D9
:10470000204698470720A560E060082231462046F1
:10471000FEF7B2FCFBF7EEFC02460E482C302434C8
:1047200000E0084601680029FBD1046000202060F9
:104730001046FBF7E3FC002070BD000013050000ED
:104740001D5200086261636B656E64006E616D6589
:1047500000000000AC040020756C6F672E696E6964
:10476000745F6F6B000000006261636B656E642DA7
:104770003E6F75747075740010B500F0EFF806495F
:1047800004484861012205A10348FFF791FF00207A
:1047900010BD0000A5470008E8050020636F6E7398
:1047A0006F6C650010B50298FDF7B6FB10BD0000F8
:1047B000FFB581B00E46040005D1FF2201325449F5
:1047C00054A0FDF7FFF9072E05D9FF220232504908
:1047D00052A0FDF7F7F90398002805D1FF22033214
:1047E0004B4954A0FDF7EEF90A98002805D1FF22A5
:1047F0000432474950A0FDF7E5F9514D00202860EB
:1048000050A0FEF731FC424FB6002C3F6860B8590B
:10481000002828680DD021184BA200F01DF9296846
:1048200040182860BA59211800F016F92968401874
:1048300028605B212154FFF7FBF801462868201807
:10484000401C00F02FF90146E86028685D224118FD
:1048500009194A7000228A702018FEF705FC2968A1
:104860003AA240182118286000F0F6F8296840188C
:10487000274928604C398A59211800F0EDF8296839
:10488000401828602118039A00F0E6F8296830A241
:1048900040182118286000F0DFF8296840182860C7
:1048A0008021091A20180B9B0A9AFFF70DFBA860BC
:1048B00029680918802903D8002801DB296002E053
:1048C00080200146286068680918491D802903D99D
:1048D0007C21081A401E28600498002807D0286808
:1048E00018A2211800F0B8F8296840182860B859B3
:1048F000002807D0286817A2211800F0ADF8296811
:104900004018286028680021215405B0F0BD00003F
:10491000EC5100086C6F675F627566006C657665C8
:104920006C203C3D204C4F475F4C564C5F44424707
:104930000000000074616700666F726D61740000B2
:10494000DC0000200D0A00001B5B000020000000BE
:104950003A2000001B5B306D0000000010B5094CD0
:104960002068002801D0002010BD0648012206A1C1
:104970000830FDF777FD0121024800226160C26224
:104980002160F0E7AC040020756C6F670000000048
:104990000FB408B506AB0093059B00F09DF801B07D
:1049A00008BC04B018470000FFB5284883B0006871
:1049B000002829D02548C56A002D22D00398800000
:1049C00002902C46243CE1680398814239D3266A40
:1049D000002E09D006980C990090019103AF0ECFDC
:1049E0002046B04700282CD0A068059908430DD078
:1049F00006980C990090019103AF0ECF204666698E
:104A00001EE00698FDF7A6FB07B0F0BD104802991E
:104A1000069F40580C9E00280CD0FEF725FB009006
:104A2000002807D00BA0FEF71FFB009940183F1885
:104A3000361A361F0097019603A90EC966692046EB
:104A4000B0472D68002DBCD1DEE70000AC0400208B
:104A5000C05100081B5B0000F8B50D000646144667
:104A6000174604D192220C490CA0FDF7ABF8002C9C
:104A70000CD1932208490AA0FDF7A4F806E03146BC
:104A8000761C802905D22870641C6D1C20780028B3
:104A9000F5D1E01BF8BD0000E0510008647374001C
:104AA0007372630070B50A46054600260A21104657
:104AB000FBF78CFB3031A955761C0200F6D1A855C6
:104AC000741E05E0295C2A5D2A542955401C641E89
:104AD000A042F7D3304670BDFFB583B00C9D1C4695
:104AE00016460F0005D18D229200214921A0FDF725
:104AF00069F8002C04D1204A1D4920A0FDF762F876
:104B00000398072805D91C4A1949921C1DA0FDF7D6
:104B100059F822480068002828D0FCF729F80290AC
:104B2000FCF7DEFE1E4829460269012A14D0012244
:104B300002610546019133463A4600940399029872
:104B4000FFF736FE009000223946029B0398FBF7E0
:104B5000AEFD0020286107E02046FDF7E9FA012EAE
:104B600002D110A0FDF7E4FAFCF7D6FE07B0F0BDC5
:104B7000FA5100087461670035020000666F726DBB
:104B8000617400006C6576656C203C3D204C4F479D
:104B90005F4C564C5F44424700000000AC040020CC
:104BA000DC0000200D0A000010B5FEF705FA002019
:104BB00010BD5F6D73685F657865635F636D6400EA
:104BC00072745F72696E676275666665725F696E40
:104BD00069740072745F72696E6762756666657289
:104BE0005F707574636861720072745F72696E677A
:104BF0006275666665725F67657463686172006698
:104C0000696E73685F6765745F70726F6D70745FF3
:104C10006D6F64650066696E73685F7365745F705D
:104C2000726F6D70745F6D6F64650066696E736836
:104C30005F7365745F6563686F0066696E73685F54
:104C40006765745F6563686F0072745F6170706C34
:104C500069636174696F6E5F696E69740072745F15
:104C60007468726561645F69646C655F65786375BB
:104C700074650072745F73656D5F696E697400724C
:104C8000745F73656D5F6465746163680072745FFF
:104C900073656D5F6372656174650072745F7365DF
:104CA0006D5F64656C6574650072745F73656D5FDC
:104CB00074616B650072745F73656D5F72656C65BE
:104CC0006173650072745F73656D5F636F6E74729C
:104CD0006F6C0072745F6D757465785F696E69746E
:104CE0000072745F6D757465785F64657461636884
:104CF0000072745F6D757465785F63726561746569
:104D00000072745F6D757465785F64656C65746559
:104D10000072745F6D757465785F74616B650072A5
:104D2000745F6D757465785F72656C65617365003D
:104D300072745F6D757465785F636F6E74726F6C9B
:104D40000072745F6576656E745F696E6974007277
:104D5000745F6576656E745F646574616368007224
:104D6000745F6576656E745F637265617465007209
:104D7000745F6576656E745F64656C6574650072FA
:104D8000745F6576656E745F73656E640072745FE0
:104D90006576656E745F726563760072745F6576C2
:104DA000656E745F636F6E74726F6C0072745F6DAA
:104DB000625F696E69740072745F6D625F646574CE
:104DC0006163680072745F6D625F637265617465D0
:104DD0000072745F6D625F64656C65746500727407
:104DE0005F6D625F73656E645F7761697400727492
:104DF0005F6D625F726563760072745F6D625F63A0
:104E00006F6E74726F6C0072745F6D715F696E6942
:104E1000740072745F6D715F6465746163680072C1
:104E2000745F6D715F6372656174650072745F6D4C
:104E3000715F64656C6574650072745F6D715F733A
:104E4000656E645F776169740072745F6D715F7520
:104E50007267656E740072745F6D715F7265637600
:104E60000072745F6D715F636F6E74726F6C0000BF
:104E70000001000200010003000100020001000423
:104E80000001000200010003000100020001000512
:104E90000001000200010003000100020001000403
:104EA00000010002000100030001000200010006F1
:104EB00000010002000100030001000200010004E3
:104EC00000010002000100030001000200010005D2
:104ED00000010002000100030001000200010004C3
:104EE00000010002000100030001000200010007B0
:104EF00000010002000100030001000200010004A3
:104F00000001000200010003000100020001000591
:104F10000001000200010003000100020001000482
:104F20000001000200010003000100020001000670
:104F30000001000200010003000100020001000462
:104F40000001000200010003000100020001000551
:104F50000001000200010003000100020001000442
:104F60000001000200010003000100020001003006
:104F700031323334353637383961626364656600FF
:104F8000303132333435363738394142434445467F
:104F90000072745F6672656500706C75675F686F3C
:104FA0006C65730072745F73797374656D5F6865A7
:104FB00061705F696E69740072745F6D616C6C6FB3
:104FC000630072745F7265616C6C6F630072745F12
:104FD0006F626A6563745F696E69740072745F6F93
:104FE000626A6563745F6465746163680072745FAC
:104FF0006F626A6563745F616C6C6F636174650096
:1050000072745F6F626A6563745F64656C65746512
:105010000072745F6F626A6563745F69735F73794E
:105020007374656D6F626A6563740072745F6F623A
:105030006A6563745F6765745F7479706500727424
:105040005F6F626A6563745F66696E640072745F45
:105050007363686564756C655F696E736572745FB0
:105060007468726561640072745F73636865647507
:105070006C655F72656D6F76655F7468726561649B
:10508000005F72745F7468726561645F696E6974F1
:105090000072745F7468726561645F696E69740040
:1050A00072745F7468726561645F73746172747541
:1050B000700072745F7468726561645F64657461C6
:1050C00063680072745F7468726561645F64656CC4
:1050D0006574650072745F7468726561645F736C97
:1050E0006565700072745F7468726561645F6465A1
:1050F0006C61795F756E74696C0072745F7468724C
:105100006561645F636F6E74726F6C0072745F745C
:1051100068726561645F73757370656E6400727444
:105120005F7468726561645F726573756D65007246
:10513000745F7468726561645F74696D656F7574BE
:105140000072745F74696D65725F696E6974007274
:10515000745F74696D65725F646574616368007221
:10516000745F74696D65725F64656C657465007207
:10517000745F74696D65725F7374617274007274C8
:105180005F74696D65725F73746F700072745F74C1
:10519000696D65725F636F6E74726F6C0000000002
:1051A000985400080000000000000000A05400080F
:1051B000A854000800000000A45400089C540008F3
:1051C000B85400080000000000000000AC540008C3
:1051D000B454000800000000B054000800000000B3
:1051E000756C6F675F73747263707900756C6F674D
:1051F0005F666F726D6174657200756C6F675F7664
:105200006F757470757400756C6F675F726177008D
:10521000756C6F675F68657864756D7000756C6F2D
:10522000675F6261636B656E645F72656769737403
:10523000657200756C6F675F6261636B656E645F5A
:10524000756E726567697374657200756C6F675F00
:105250006261636B656E645F7365745F66696C74CD
:10526000657200756C6F675F6261636B656E645F2A
:1052700066696E640000000001000000020000008A
:1052800004000000080000001000000020000000E2
:105290004000000080000000252D2A2E732070722F
:1052A000692020737461747573202020202020737E
:1052B000702020202020737461636B2073697A65ED
:1052C000206D61782075736564206C656674207448
:1052D00069636B20206572726F720A0072745F6F6F
:1052E000626A6563745F6765745F747970652826A8
:1052F00073656D2D3E706172656E742E706172659E
:105300006E7429203D3D2052545F4F626A6563747C
:105310005F436C6173735F53656D6170686F726535
:105320000000000072745F6F626A6563745F676596
:10533000745F7479706528266D757465782D3E707C
:105340006172656E742E706172656E7429203D3DC8
:105350002052545F4F626A6563745F436C6173737C
:105360005F4D7574657800002872745F75626173B3
:10537000655F7429282872745F75696E74385F746C
:10538000202A296D656D202B2053495A454F465FD1
:105390005354525543545F4D454D292025205254B6
:1053A0005F414C49474E5F53495A45203D3D2030AF
:1053B000000000002872745F75696E74385F742095
:1053C0002A29726D656D203E3D202872745F7569D3
:1053D0006E74385F74202A29686561705F7074721A
:1053E000202626202872745F75696E74385F7420D9
:1053F0002A29726D656D203C202872745F75696E74
:1054000074385F74202A29686561705F656E640076
:105410002872745F75626173655F74296D656D20B4
:105420002B2053495A454F465F5354525543545FBE
:105430004D454D202B2073697A65203C3D20287214
:10544000745F75626173655F7429686561705F651B
:105450006E64000072745F6F626A6563745F676593
:10546000745F74797065282872745F6F626A65630F
:10547000745F742974687265616429203D3D20520F
:10548000545F4F626A6563745F436C6173735F540A
:105490006872656164000000412F0000442F000025
:1054A000452F0000492F0000572F000033316D00B9
:1054B00033326D0033336D0033356D0068656C6CCD
:1054C0006F007361792068656C6C6F20776F726C08
:1054D000640076657273696F6E0073686F7720522F
:1054E000542D5468726561642076657273696F6EBD
:1054F00020696E666F726D6174696F6E005F5F63C5
:105500006D645F76657273696F6E0073686F772084
:1055100052542D5468726561642076657273696FA8
:105520006E20696E666F726D6174696F6E006C6972
:1055300073745F746872656164006C69737420745D
:105540006872656164005F5F636D645F6C6973744A
:105550005F746872656164006C697374207468724A
:10556000656164006C6973745F73656D006C697369
:10557000742073656D6170686F726520696E207349
:10558000797374656D005F5F636D645F6C697374DC
:105590005F73656D006C6973742073656D6170680D
:1055A0006F726520696E2073797374656D006C6924
:1055B00073745F6576656E74006C697374206576CC
:1055C000656E7420696E2073797374656D005F5F1A
:1055D000636D645F6C6973745F6576656E74006C8F
:1055E000697374206576656E7420696E20737973B3
:1055F00074656D006C6973745F6D75746578006CAB
:10560000697374206D7574657820696E2073797381
:1056100074656D005F5F636D645F6C6973745F6D6B
:1056200075746578006C697374206D757465782085
:10563000696E2073797374656D006C6973745F6D46
:1056400061696C626F78006C697374206D61696C5C
:1056500020626F7820696E2073797374656D005FC6
:105660005F636D645F6C6973745F6D61696C626FB9
:1056700078006C697374206D61696C20626F7820AA
:10568000696E2073797374656D006C6973745F6DF6
:1056900073677175657565006C697374206D6573EA
:1056A0007361676520717565756520696E20737912
:1056B0007374656D005F5F636D645F6C6973745FC5
:1056C0006D73677175657565006C697374206D65C0
:1056D000737361676520717565756520696E2073E8
:1056E000797374656D006C6973745F74696D65724C
:1056F000006C6973742074696D657220696E207323
:10570000797374656D005F5F636D645F6C6973745A
:105710005F74696D6572006C6973742074696D657E
:105720007220696E2073797374656D006C6973748F
:10573000006C69737420616C6C2073796D626F6C9E
:1057400020696E2073797374656D005F5F636D64AB
:105750005F68656C700052542D54687265616420F6
:105760007368656C6C2068656C702E005F5F636D9C
:10577000645F7073004C697374207468726561644F
:105780007320696E207468652073797374656D2E5B
:10579000005F5F636D645F667265650053686F7775
:1057A00020746865206D656D6F727920757361670F
:1057B0006520696E207468652073797374656D2E39
:1057C000006C6973745F6D656D006C697374206D36
:1057D000656D6F727920757361676520696E666F9C
:1057E000726D6174696F6E004941000841410008A3
:1057F0005D4900083D41000879470008A1070008FD
:1058000045410008BC540008C2540008890B000838
:10581000D2540008DA540008A94B0008FD540008CF
:105820000B550008A94B00082E5500083A550008F2
:10583000ED1200084655000858550008ED12000802
:10584000645500086D550008D11100088655000800
:1058500095550008D1110008AE550008B95500084B
:105860004D0C0008CE550008DF5500084D0C00080F
:10587000F4550008FF550008D91000081456000818
:1058800025560008D91000083A5600084756000867
:10589000090E00085F56000872560008090E00083D
:1058A0008A56000898560008B10F0008B55600083F
:1058B000C9560008B10F0008E6560008F156000866
:1058C000AD1400080657000817570008AD1400086B
:1058D0002C57000831570008E90B00084B57000807
:1058E000565700087D1700086C57000875570008C8
:1058F000A5060008915700089C5700089B06000861
:10590000C1570008CA570008450F00082C59000865
:1059100000000020F8000000A8040008245A000835
:10592000F800002058090000B8040008000000003A
:105930000000000000000000000000000000000067
:105940000000000000000000000000000000000057
:105950000000000000000000000000000000000047
:105960000000000000000000000000000000000037
:1059700000000000000000000100000050000020B6
:1059800050000020800000000200000060000020A5
:1059900060000020200000000300000070000020D4
:1059A000700000202400000004000000800000209F
:1059B0008000002020000000050000009000002072
:1059C000900000203000000006000000A000002031
:1059D000A00000203C0000000A000000B0000020F1
:1059E000B00000202C0000000000000000000000BB
:1059F00000000000000000000000000000000000A7
:105A00000000000000000000000000000000000096
:105A10000000000000000000000000000000000086
:045A20000024F4006A
:04000005080000C12E
:00000001FF
